:10000000E9C022C079C091C096C09BC006C09FC005
:1000100019C0CFC018C0D3C0D8C0A8957F938F9304
:100020008FB779B77D7779BF7DEF7DBD79EA7CBDEC
:1000300071E07093720079B7726879BF8FBF8F914A
:100040007F911895189518950F937F939F938F9391
:100050008FB77BB77F7B7BBF00E000939B007091E5
:100060008C007A9570938C0070918B007A9570302B
:1000700009F47AE070938B0070919400703009F469
:1000800003C07A957093940072E070937200B09BF5
:1000900011C070917100713039F490918D009030E1
:1000A00011F100E1009372007030C9F490E0909378
:1000B0008D0019C070917100773039F490918D00E6
:1000C000903089F401E100937200783021F49FEFC1
:1000D00090938D0008C073957093710004C07A9559
:1000E0007093710000C07BB770647BBF8FBF8F912E
:1000F0009F917F910F9118957F938F938FB77BB7C7
:100100007F777BBF70918D00703041F470919B00C0
:10011000739570939B0072E0709372007BB7706868
:100120007BBF8FBF8F917F9118958FB779B7777FFE
:1001300079BF8FBF18958FB779B77F7B79BF8FBF96
:1001400018958FB779B77F7D79BF8FBF1895A89520
:100150007F938F939F938FB770919A0072BF70E0D7
:100160007093730090918D009F3FF1F0B29B03C09C
:10017000B39B07C016C0B39B08C071E270937300B5
:1001800008C072E27093730004C073E2709373004E
:1001900000C070918C007F3F09F0739570938C00C4
:1001A00003C070E070938C008FBF9F918F917F91FF
:1001B00018958FB70F930CB10F918FBF18958FB70C
:1001C0007AB17F7B7AB98FBF18958FB773E878B90A
:1001D0008FBF18950FE101BD0FE50DBF02E00EBF07
:1001E00000E007BB01BB0FEF08BB02BBEFEFEABBB0
:1001F000E4BBEE27EBBBE5BBAD9AA89A00E00ABFD3
:10020000AC9AD6D6AC9800E009BF0FB700600FBF1C
:1002100000000000000000000000000000000000DE
:1002200000000FB70F770FBF00E009BF00E00BBF62
:1002300000E908B90EE005BF05E003BF01E0009347
:100240009A0000919A0002BF00E00FBD07E00EBDCA
:100250007DEF7DBD79EA7CBD00EC0BBF00E009BFFE
:1002600009B7026809BF0FB700680FBFEBD77BD58E
:1002700081D741E04093940006C3B7D5A1E048EB95
:1002800077D640E075D6DFE0C0ED91D530917300B0
:10029000313209F406C0323209F416C03332B9F5EE
:1002A00026C086D6009197000395077000939700AB
:1002B000A1E048EB5DD640E45BD64091970056D66E
:1002C00030E03093730023C073D6009196000395FD
:1002D000077000939600A1E048EB4AD644E448D664
:1002E0004091960043D630E03093730010C060D642
:1002F00030E03093730000919700109196001295B2
:10030000102B163709F40AC0153211F41FC1BECFE5
:1003100000E00093970000939600AFCF00E00093B9
:1003200097000093960000E0009398005ED5A1E04E
:1003300049EB1ED640E01CD6DFE0CAED38D566E0BA
:10034000F0E0E0E652E095D710C0A1E04AEB10D60D
:1003500040E0C6D430917300313209F406C0323225
:1003600009F410C0333289F724C022D6DED00091C0
:1003700098000395077000939800C6D030E0309342
:100380007300E3CF15D6009198000030D9F001300A
:10039000D1F00230C9F00330C1F00430B9F00530BB
:1003A000B1F00630A9F00730A1F030E030937300CF
:1003B000CCCF66E0F0E0E0E652E061D730E0309389
:1003C000730061C207C01AC02BC03EC04FC062C0DC
:1003D00073C086C000916200109162001F70029588
:1003E0000F70023028F000E0102B109362008AC0DA
:1003F00003950295102B1093620084C00091620057
:1004000010916200107F0F70093028F000E0102B6F
:100410001093620077C00395102B1093620072C096
:1004200000916100109161001F7002950F700530FE
:1004300028F000E0102B1093610064C00395029532
:10044000102B109361005EC000916100109161005B
:10045000107F0F70093028F000E0102B109361001E
:1004600051C00395102B109361004CC000916300A4
:10047000109163001F7002950F70033028F000E0A8
:10048000102B109363003EC003950295102B109320
:10049000630038C00091630010916300107F0F70FB
:1004A000093028F000E0102B109363002BC0039557
:1004B000102B1093630026C000916400109164001B
:1004C0001F7002950F70013028F000E0102B109380
:1004D000640018C003950295102B1093640012C09D
:1004E0000091640010916400107F0F70093028F0B3
:1004F00000E0102B1093640005C00395102B10939F
:10050000640000C022CFFFCF4BEB32D52091980082
:1005100030E0F6E0E6E5E20FF31FC895402D28D560
:10052000F6E0E6E417E03BD408954BEB21D52091AB
:10053000980030E0F6E0E6E5E20FF31FC895402DA5
:1005400017D5F6E0EEE417E02AD4089500E0009312
:1005500097000093960049D4A1E048EB09D540E00C
:1005600007D5D6E0CEE523D4A1E049EB01D540E0A4
:10057000FFD4D6E0CEE61BD430917300313209F4BB
:1005800006C0323209F413C03332B1F720C010D59F
:10059000A1E049EBEDD440E0EBD4D6E0CEE607D4C1
:1005A00007E30093990030E030937300E5CF00D566
:1005B000A1E049EBDDD440E0DBD4D6E0C6E6F7D3DA
:1005C00000E00093990030E030937300D5CF0091A4
:1005D00099000030A1F500E00093750000937400CD
:1005E000009379000093780000937F0000938000CF
:1005F00042D000E0502F602F402F5F936F93A1E017
:1006000048EBB6D446E4B4D4452FB0D4A1E048EBCF
:10061000AFD444E4ADD4462FA9D46F915F9140E0AC
:100620005F936F9332D671D46F915F9121E030E088
:100630008894520F631F062F052B0030F1F630E02F
:100640003093730020C1000C0E0F0E0C0000000050
:1006500000000000000000060F152D333C42636CC3
:100660006561723F000079657300000000006E6FE5
:1006700020000000000050E440917500E7D553953C
:1006800040917400E3D5539540917F00DFD5539599
:1006900040918000DBD5089505B7006205BFAA9A96
:1006A0008895AA980091720030917300013109F485
:1006B0003BC2003109F4E6C010918D00103049F4BE
:1006C000313209F44AC2323209F459C2333221F4C8
:1006D00071C2023009F448C0013009F407C030E0AB
:1006E0003093730000E0009372007BC000E0009341
:1006F0007200A1E048EB3CD440E03AD4C0917F00C6
:10070000D09180002196C0937F00D09380000C2F61
:100710001D2FD2D5DBD2F9E1E8E764D3A1E048EBA5
:1007200027D448E225D4C0917D00D0917E00219647
:10073000C0937D00D0937E000C2F1D2FBDD5C6D257
:1007400050C01F932F933F9312951F70022F229535
:10075000207F122B202F22952F703295307F232B54
:100760003F912F911F91089500E00093720080D374
:1007700058EB38D259EB36D25AEB34D25BEB32D24B
:100780000091900000938E000091910000938F00E3
:100790000CB5009390000DB50093910030918E0040
:1007A00040918F0050919000609191008894531B6C
:1007B000640BA0F0052F162F26E030E01ED4009326
:1007C000920000938900083108F008E1B02E21E082
:1007D000922E2EE4822EA22E26D403C000919200E7
:1007E000F2CF10918D00103039F400919B00003051
:1007F00011F034D001C03CD03EDF009194000030B5
:1008000051F466E0F0E0E0E652E033D5A0E048EBDA
:10081000AFD348E065D210918D00103011F405D2AD
:100820003BCFF7D1609175005091740000918B001F
:10083000013099F40AE000938B004091890025D59E
:10084000609175005091740040E031E08894530F3E
:10085000641F60937500509374001ECFA0E048EBB6
:1008600087D341E085D3FBE1E8EF19E098D2089502
:10087000A0E048EB7DD341E07BD3FBE1E0EF19E062
:100880008ED20895E6D100E000937200AED212D26B
:1008900060917700509176006093790050937800D2
:1008A0000FE90093930004D000E00093720099CF09
:1008B00035D06091790050917800F1D44F9390D069
:1008C0004F9147FD0BC0042F083108F008E1B02E0E
:1008D00020E0922E2FE4822EA22EA5D360917500E7
:1008E0005091740040917900309178008894531BA6
:1008F000640B609179005091780040E031E0889479
:10090000530F641F60937900509378000091930017
:100910000A9519F000939300CBCF08956091790068
:100920005091780040E03EE48894531B640BB7D4A8
:1009300047FF36C00091950007FF0BC006FF0DC0B2
:1009400005FF12C004FF17C003FF1CC002FF21C037
:1009500024C04F3F11F5006820C047FF1EC000644F
:100960004F7740936A0019C047FF17C000624F7766
:100970004093690012C047FF10C000614F77409359
:100980006B000BC047FF09C008604F7740936C00B5
:1009900004C0403F11F4046007C00093950008951F
:1009A00000E0009395000895A1E04BEBE1D24FE405
:1009B000DFD245E5DBD24AEBDBD24FE4D9D245E5C5
:1009C000D5D249EBD5D24FE4D3D245E5CFD2A0E082
:1009D00048EB15D249E0A4D100E0009395000895BA
:1009E00047D259EBFFD05AEBFDD05BEBFBD008951B
:1009F0002FD0609179005091780040E03FE98894D1
:100A0000531B640B4CD44F9385D04F9147FD0BC0C3
:100A1000042F083108F008E1B02E20E0922E21E0EA
:100A2000822EA22E00D3609179005091780040E090
:100A300031E08894531B640B6093790050937800E5
:100A4000009193000A9519F000939300D1CF089577
:100A5000609179005091780040E035E58894531B0F
:100A6000640B1DD447FF36C00091950007FF0BC0F3
:100A700006FF0DC005FF12C004FF17C003FF1CC016
:100A800002FF21C024C0403F11F5006820C047FF8D
:100A90001EC000644F7740936C0019C047FF17C019
:100AA00000624F7740936B0012C047FF10C0006197
:100AB0004F77409369000BC047FF09C008604F772C
:100AC00040936A0004C04F3F11F4046007C00093D4
:100AD0009500089500E0009395000895A1E04BEB88
:100AE00047D24DE445D245E541D24AEB41D24DE4EF
:100AF0003FD245E53BD249EB3BD24DE439D245E507
:100B000035D2A0E048EB7BD149E00AD100E0009368
:100B100095000895D0D158EB5DD059EB5BD05AEBDE
:100B200059D05BEB57D0089500E000937D0000930F
:100B30007E0060917500509174006093770050932F
:100B400076007FD000E0009372004FD105E0009363
:100B50008B0000E00093720044CE00E0009372002E
:100B6000609179005091780001E000939300A0DE3D
:100B700030E03093730000E00093720027C0609172
:100B800079005091780040E03FE98894531B640B52
:100B900000E000937200609179005091780001E0CC
:100BA0000093930025DF30E03093730000E0009362
:100BB00072000CC000918C00003308F05ECB30E076
:100BC0003093730000E00093720000C007E00093D0
:100BD000940062CDA1E0452FCBD140E0C9D140E0E7
:100BE000C5D10895A0E0452FC3D14FE4C1D140E065
:100BF000BDD1089559EB05D05AEB03D05BEB01D082
:100C00000895A0E0452FB4D14FE4B2D145E5AED16F
:100C100008950F93A1E048EBABD146E4A9D1FBE1E5
:100C2000E8EE18E0BCD00F9108950F93A1E048EBD7
:100C30009FD146E49DD1FBE1E0EF18E0B0D00F91E9
:100C4000089540E022D04FEF20D00BD040EF1DD0D0
:100C5000089540E01AD04FEF18D003D040EF15D0E0
:100C60000895409162004F7340680FD04091610039
:100C700040680BD0409163004F73406806D04091AC
:100C800064004F71406801D00895609175005091E3
:100C90007400FBD23AD139D1609175005091740043
:100CA00040E031E08894530F641F609375005093C7
:100CB00074000895A1E048EB5BD14DE459D140E4C4
:100CC00055D14FEF53D140E451D108951F932F9345
:100CD0003F934F914ED04F914CD04F914AD00895B1
:100CE00047D1409162004F7344D0F9E1E0ED7AD0F2
:100CF000409161003ED0F9E1E0ED74D04091600098
:100D000038D0F9E1E0E06ED0409163004F7331D00C
:100D1000F9E1E0E767D0409164004F712AD008956F
:100D200027D140916A004F7324D0F9E1E0ED5AD009
:100D3000409169001ED0F9E1E0E054D0F9E1E0E033
:100D400051D0F9E1E0E04ED0F9E1E0E04BD0409144
:100D50006B004F730ED0F9E1E0E744D040916C0096
:100D60004F7107D00895A0E0C9D0A1E0C7D03DD011
:100D700008954F9342954F7004D04F914F7001D01A
:100D80000895242FF9E1E0E830E08894220F331F22
:100D9000220F331F220F331FE20FF31F17E0C895F6
:100DA0001A9521F0402DE2D03196F9CF0895EC2F1D
:100DB000FD2FC895202D203021F0202D03D0219625
:100DC000F6CF0895F8E1E0E030E08894220F331F79
:100DD000220F331F220F331F8894E20FF31F17E0F7
:100DE000DEDF089514E0DBDF0895A1E001D0A0E08C
:100DF00048EB05D049EB03D04AEB01D04BEBB8D020
:100E000040E0B6D050E840E0B1D05A95E1F70895FF
:100E1000A0E049EBADD007D04AEBAAD004D04BEB11
:100E2000A7D001D008956EE4462FA2D079D0462FE6
:100E300043959ED0432D9AD06A956F3FA9F70895A8
:100E4000A0E049EB95D007D04AEB92D004D04BEB11
:100E50008FD001D0089561E0462F8AD061D0462F0F
:100E60004A9586D0432D82D063956035A9F70895C1
:100E7000A1E009D069EB11D06AEB0FD06BEB0DD07C
:100E8000A0E001D0089549EB73D0E5DF4AEB70D0C4
:100E9000E2DF4BEB6DD0DFDF0895A0E0462F68D096
:100EA00040E066D03DD0A1E0462F62D04FE460D054
:100EB000432D5CD00895A0E009D069EB11D06AEB16
:100EC0000FD06BEB0DD0A1E001D0089549EB50D0CD
:100ED000AADF4AEB4DD0A7DF4BEB4AD0A4DF089541
:100EE000A1E0462F45D04FE443D01AD0A0E0462FD2
:100EF0003FD040E03DD0432D39D008954FEA38D05F
:100F000008952FEF2A95F1F708952F933F932FEF30
:100F10003FEF3A95F1F72A95E1F73F912F91089528
:100F200000E00ABB0FEF0BBBAE9AA03069F0A898A7
:100F3000AB9AA9980000A99A0000A998000039B2BC
:100F40000000AB98A89A0CC0AD98AB9AA998000085
:100F5000A99A0000A998000039B20000AB98AD9A98
:100F6000A99A00E00BBB0FEF0ABB0895AE9A03C02D
:100F7000AE9801D008954BBB00000000A03061F096
:100F8000A898AB980000A99800000000000000009D
:100F9000A99AAB9AA89A0895AD98AB980000A99821
:100FA0000000000000000000A99AAB9AAD9A0895D5
:100FB0001F932F933F9314E12FEF3FEF3A95F1F7F3
:100FC0002A95E1F71A95D1F73F912F911F91089536
:100FD000706173776F72643A000073657420636C9C
:100FE0006F636B3A0000222738E0169508F4200F53
:100FF000279517953A95D1F70895EE24FF1841E10A
:10100000001F111F4A9509F40895EE1CFF1CE21AF7
:10101000F30A20F4E20EF31E8894F2CF0894F0CF86
:1010200037C067C06DC0CA2CC818E1F3DB2CD918D3
:10103000C1F3B0F30C2D0D15B4F4792D91E00C2D06
:10104000192FD1DF012F122F2D2D30E0D6DF802F69
:10105000082D080F602F7B1529F000C066D073950E
:101060009395EDCF82C0682D81E00D2D182FBBDF49
:10107000012F122F2C2D30E0C0DF902F092D090FEA
:10108000702F6A1579F300C050D063958395EDCF2A
:10109000D92CDB180C2D0D15B4F4792D91E00C2D05
:1010A000192FA1DF012F122F2D2D30E0A6DF802F69
:1010B000082D080F602F7B1529F000C036D07A95D7
:1010C0009395EDCF52C0682D81E00D2D182F8BDF49
:1010D000012F122F2C2D30E090DF902F092D091BAE
:1010E000702F6A1529F000C020D063958395EDCF4D
:1010F0003CC0682D792D19D06395A616E1F735C04F
:10110000B91440F071F0682D792D0FD07395B71692
:10111000E1F72BC0682D792D08D07A95B716E1F745
:1011200024C0682D792D01D020C00FE1502E571A10
:10113000552D052D0770502E56955695569508EB52
:10114000500FF1E1ECE66624E50DF61DC895502C34
:10115000452F0EDF462F0CDFE3DE3528452F08DF55
:10116000462F06DF432D02DF08950895010204088B
:101170001020408002E00093710000E00093950091
:1011800050E46CD04093750040937700539566D03F
:101190004093740040937600539560D040937F0055
:1011A00053955CD0409380005395089502E00A95D2
:1011B000F1F7089501E00A95F1F708958C9A8D985A
:1011C000F5DF8C98F7DF122F8D9AF4DF0894111F4A
:1011D00001C0110F59F08C9A18F400008D9802C0CC
:1011E0008D9A00C0E3DF8C98E1DFF3CF8C9A8D9865
:1011F000DDDF8C98849BFECF889485990894D6DF98
:10120000089520FFE3CF331F11E08C9ACFDF8C9835
:10121000CDDF889485990894111FB8F78C9A37957B
:1012200010F48D9801C08D9AC1DF8C98849BFECFFD
:10123000BDDF08958C9A8D9AB9DF8C98BBDF8D98AD
:10124000B5DF0895332732BB31BB089520EABBDFF9
:10125000152FD7DF142FD5DFEDDF089520EAB3DF98
:10126000152FCFDF21EAAADF0894CBDFE3DF412F80
:101270000895F4DF419353956A95D9F70895419104
:10128000E5DF53956A95D9F7089522EA9CDF162F7A
:10129000B8DF152FB6DF142FB4DFCCDF089522EAB4
:1012A00092DF162FAEDF152FACDF23EA87DF08941D
:1012B000A8DFC0DF412F08953FEF3395005117425B
:1012C000E0F7005F184D2FEE205F085E1340E0F757
:1012D00008511C4F239504561040E0F70C5910EFAD
:0C12E000105F0A50E8F7065F100F089539
:081900000000000000000000DF
:101970000060600000000000002010080402010068
:10198000003E5149453E00000000427F40000000FB
:101990000042615149460000002141454B310000A1
:1019A000001814127F10000000274545453800003C
:1019B000003C4A494930000000017109050300005C
:1019C000003649494936000000064949291E0000F1
:0819D0000036360000000000A3
:0819F800000201510906000084
:101B08000020545454780000007F484444380000B2
:101B1800003844444420000000384444487F000012
:101B2800003854545418000000087E0901020000CF
:101B380000085454543C0000007F08040478000056
:101B48000000447D40000000002040443D000000AB
:101B5800007F1028440000000000417F4000000082
:101B6800007C041804780000007C08040478000055
:101B78000038444444380000007C14141408000061
:101B880000081414147C0000007C080404080000F9
:101B9800004854545420000000043F4440200000F2
:101BA800003C4040207C0000001C2040201C00001D
:101BB800003C403C403C0000004428102844000001
:101BC800000C5050503C0000004464544C44000049
:101BD8000000FE03FE0000001C3E3FFEBF3E1C004E
:101BE80000007F384CFE40000000000000000000AC
:101BF80040784EC3C34E78402D4156544F494E4607
:101C08004F2056332E30204156522D0000005935B2
:061C18001231060000007D
:00000001FF
